:100000000C9444000C946C000C946C000C946C00E8
:100010000C946C000C946C000C946C000C946C00B0
:100020000C946C000C946C000C946C000C946701A4
:100030000C946C000C946C000C946C000C946C0090
:100040000C946C000C946C000C94F0030C946C00F9
:100050000C946C000C946C000C946C000C946C0070
:100060000C946C000C946C0005A84CCDB2D44EB925
:100070003836A9020C50B9918688083CA6AAAA2A4B
:10008000BE000000803FCE0111241FBECFEFD8E09C
:10009000DEBFCDBF11E0A0E0B1E0ECE7F6E102C0C9
:1000A00005900D92AA32B107D9F713E0AAE2B1E0A8
:1000B00001C01D92A43BB107E1F710E0C8E8D0E011
:1000C00004C02297FE010E94A309C638D107C9F7D0
:1000D0000E94FE000C943C0B0C940000DF93CF9325
:1000E000CDB7DEB764970FB6F894DEBF0FBECDBFB5
:1000F00088ED9FE0A9E4B0E48F839887A987BA8749
:1001000080E090E0DC0189839A83AB83BC832F81FC
:10011000388549855A85CA01B9010E947705DC01F5
:10012000CB01BC01CD0120E030E040E054E40E946E
:10013000CF06DC01CB018B879C87AD87BE871E82F3
:100140001D8248C089819A81AB81BC81BC01CD01EF
:100150000E94A709DC01CB01BC01CD0120E030E009
:100160004EEF52E40E94D505DC01CB018F87988BBE
:10017000A98BBA8B69817A818B819C812B853C8587
:100180004D855E850E947705DC01CB0189839A83CA
:10019000AB83BC836F85788989899A8920E030E0B8
:1001A00040E053E40E947705DC01CB01BC01CD01A6
:1001B0000E947D07DC01CB019C8B8B8B2B898D8171
:1001C0009E81865D9E4FFC0120838D819E810196DC
:1001D0009E838D8321E08D819E81F2E080309F0798
:1001E0000CF020E0222309F0ADCF64960FB6F8940E
:1001F000DEBF0FBECDBFCF91DF910895DF93CF93C8
:100200000F92CDB7DEB70E946E008EE293E040E021
:1002100052EC61E070E00E94E20184E290E024E2AE
:1002200030E0F90120812062FC01208385E290E02A
:1002300020E2FC01208381E890E021E830E0F90130
:1002400020812860FC0120838FE690E02FE630E0DB
:10025000F90120812260FC01208388E890E026E8F3
:1002600031E0FC0131832083789403C0000001C099
:1002700000008EE293E00E94DF0121E018161906CB
:100280000CF020E0222391F385E290E025E230E0BB
:10029000F901308120E22327FC0120838EE293E0E4
:1002A0000E94DC0189838981813611F78EE293E017
:1002B00020E031E0B9010E94360281E890E021E8B7
:1002C00030E0F90120812560FC012083D2CF1F920C
:1002D0000F920FB60F9211242F933F934F935F937A
:1002E0006F937F938F939F93AF93BF93EF93FF93FE
:1002F000DF93CF9300D0CDB7DEB785E290E025E263
:1003000030E0F901308120E22327FC0120831A82AA
:10031000198220C080912C0390912D03865D9E4F01
:10032000FC0120818EE293E0622F0E94D501809132
:100330002C0390912D03019620E032E0B9010E9438
:10034000060990932D0380932C0389819A8101964D
:100350009A83898321E089819A81F1E080349F0723
:100360000CF020E02223B1F68EE293E060E00E94E0
:10037000D5010F900F90CF91DF91FF91EF91BF9139
:10038000AF919F918F917F916F915F914F913F912D
:100390002F910F900FBE0F901F9018958FE191E055
:1003A00090932F0380932E030895862F0E94AF030E
:1003B00008950E94E70308950E94C80308950E94CB
:1003C000B7030895CB01BA010E9476030895DC01BA
:1003D000ED91FC910190F081E02D09950895DC01EB
:1003E000ED91FC910190F081E02D099508950F9316
:1003F0001F93CF93DF938C01EB0109C02196D801A5
:10040000ED91FC910190F081E02DC8010995688182
:100410006623A1F7DF91CF911F910F9108950F935C
:100420001F938C01DC01ED91FC910190F081E02D96
:100430006DE00995D801ED91FC910190F081E02DDE
:100440006AE0C80109951F910F9108950F931F93BA
:100450008C01DC01ED91FC910190F081E02D09957A
:10046000C8010E940F021F910F9108950F931F93CF
:100470008C010E94F701C8010E940F021F910F9189
:1004800008950F931F938C01DC01ED91FC91019075
:10049000F081E02D0995C8010E940F021F910F9174
:1004A00008952F923F924F925F926F927F928F9218
:1004B0009F92AF92BF92CF92DF92EF92FF920F93F3
:1004C0001F93DF93CF93CDB7DEB7A0970FB6F89405
:1004D000DEBF0FBECDBF1C016A017B014115510576
:1004E0006105710549F4DC01ED91FC910190F08109
:1004F000E02D60E3099554C0882499245401422ECC
:1005000055246624772401E010E00C0F1D1F080D10
:10051000191DC701B601A30192010E941909F80132
:1005200060830894811C911CA11CB11CC701B601F9
:10053000A30192010E941909C901DA016C017D0130
:10054000C114D104E104F104F1F681E0E82EF12CAC
:10055000EC0EFD1EE80CF91C3E010894611C711C98
:10056000D501C4010197A109B1096C01C818D908C6
:1005700014C0F601EE0DFF1D60816A3010F4605D5D
:1005800001C0695CD101ED91FC910190F081E02DF9
:10059000C10109950894E108F1086E147F0449F738
:1005A000A0960FB6F894DEBF0FBECDBFCF91DF91FE
:1005B0001F910F91FF90EF90DF90CF90BF90AF9081
:1005C0009F908F907F906F905F904F903F902F9073
:1005D00008952AE00E94510208950F931F938C0101
:1005E0000E94E902C8010E940F021F910F91089515
:1005F000AB0160E070E00E94E90208950F931F9341
:100600008C01AB0160E070E00E94E902C8010E9429
:100610000F021F910F910895EF92FF920F931F9376
:10062000CF93DF93EC017A018B0177FF0FC0E88154
:10063000F9810190F081E02D6DE20995109500950A
:10064000F094E094E11CF11C011D111D2AE0B80199
:10065000A701CE010E945102DF91CF911F910F910E
:10066000FF90EF9008950F931F938C010E940C034D
:10067000C8010E940F021F910F910895AB016627D8
:1006800057FD6095762F0E940C0308950F931F93DA
:100690008C01AB01662757FD6095762F0E940C03F5
:1006A000C8010E940F021F910F910895DC012115CE
:1006B000310541F4ED91FC910190F081E02D642F22
:1006C000099508952A30310519F40E940C03089504
:1006D0000E94510208950F931F938C010E945603AC
:1006E000C8010E940F021F910F910895EF92FF928F
:1006F0000F931F937B018C0122E030E040E050E03B
:100700000E943B09205C3D4B404F5F4FCA01B9013D
:10071000A80197010E943B09C901DA010197A109CB
:10072000B109292F3A2F4B2F552747FD5A9501968E
:10073000A11DB11D2093C50081508093C400E1EC40
:10074000F0E0808180618083808188608083808107
:10075000806880831F910F91FF90EF900895982FEC
:100760008091C00085FFFCCF9093C60008958091D2
:1007700030039091310380589F4F20913203309184
:100780003303821B930B60E870E00E940609089512
:1007900040913203509133038091300390913103A3
:1007A0008417950719F42FEF3FEF0FC0FA01EC5CA7
:1007B000FC4F2081CA01019660E870E00E940609A2
:1007C000909333038093320330E0C9010895809100
:1007D0003203909133039093310380933003089553
:1007E0001F920F920FB60F9211242F933F934F93A6
:1007F0005F936F937F938F939F93AF93BF93EF9389
:10080000FF934091C600E0913003F0913103CF0196
:10081000019660E870E00E9406099C018091320315
:10082000909133032817390739F0EC5CFC4F408373
:100830003093310320933003FF91EF91BF91AF913B
:100840009F918F917F916F915F914F913F912F91E8
:100850000F900FBE0F901F901895A0E0B0E0E3E35B
:10086000F4E00C946E09FC01EA018081823008F406
:1008700038C1DB019C91923008F430C1843059F4C6
:10088000943009F02EC1918111968C91119798178F
:1008900009F021C126C1943009F420C19230B1F48D
:1008A000823009F01EC1CA01AF0128E0DA010D90C3
:1008B000AD01DC010D92CD012150C1F7DB01119694
:1008C0008C9111979181892389830AC1823009F41F
:1008D00005C1C280D380DB0112966D907C90139786
:1008E00024813581468157811496ED90FD900D91BC
:1008F0001C911797C601861997095C0197FF04C0E0
:10090000AA24BB24A81AB90AB0E2AB16B1040CF0B1
:1009100061C0181619066CF5370148010A2C04C08D
:1009200096948794779467940A94D2F781E090E044
:10093000A0E0B0E00A2C04C0880F991FAA1FBB1FBB
:100940000A94D2F70197A109B1098E219F21A02312
:10095000B123EE24FF248701E3940097A105B1059C
:1009600019F4EE24FF248701E628F728082919291D
:100970003CC00097D1F1CA0CDB1C39014A010A2C9A
:1009800004C096948794779467940A94D2F781E090
:1009900090E0A0E0B0E00A2C04C0880F991FAA1FC5
:1009A000BB1F0A94D2F70197A109B10982239323AF
:1009B000A423B52321E030E040E050E00097A105FA
:1009C000B10519F420E030E0A9012629372948298A
:1009D00059290BC06C147D0424F4EE24FF248701F4
:1009E00004C0630120E030E0A9018181FB01918115
:1009F000891709F445C0882349F0D801C701821B33
:100A0000930BA40BB50B9C01AD0104C02E193F093B
:100A1000400B510B57FD04C01982DB82CA820BC008
:100A200081E08983DB82CA8250954095309521957B
:100A30003F4F4F4F5F4F2C833D834E835F830DC0ED
:100A4000880F991FAA1FBB1F8C839D83AE83BF8312
:100A50008A819B8101979B838A838C819D81AE8152
:100A6000BF819C01AD0121503040404050402F3F9C
:100A7000EFEF3E07EFEF4E07EFE35E0708F30BC023
:100A80008983DB82CA822E0D3F1D401F511F2C839C
:100A90003D834E835F8383E088832C813D814E813B
:100AA0005F8157FF1DC0DA01C90181709070A0708D
:100AB000B0705695479537952795822B932BA42B8D
:100AC000B52B8C839D83AE83BF838A819B810196E6
:100AD0009B838A8305C0E1E2F1E003C0FB0101C012
:100AE000FE01CF01CDB7DEB7EEE00C948A09A0E29B
:100AF000B0E0EDE7F5E00C94760969837A838B83A7
:100B00009C832D833E834F83588789E0E82EF12C08
:100B1000EC0EFD1ECE010196B7010E949D088E01CC
:100B20000F5E1F4FCE010596B8010E949D08C701B8
:100B3000B801AE01475E5F4F0E942D040E94CF07AF
:100B4000A096E6E00C949209A0E2B0E0EAEAF5E0B3
:100B50000C94760969837A838B839C832D833E83EF
:100B60004F8358878E01075F1F4FCE010196B80152
:100B70000E949D0891E1E92EF12CEC0EFD1ECE01A4
:100B80000596B7010E949D088A8991E089278A8B82
:100B9000C801B701AE01475E5F4F0E942D040E945D
:100BA000CF07A096E6E00C949209A0E2B0E0EBED4E
:100BB000F5E00C946A0969837A838B839C832D8387
:100BC0003E834F835887CE010196BE01675F7F4FFA
:100BD0000E949D08CE010596BE016F5E7F4F0E9468
:100BE0009D089985923078F089898230C0F09430E0
:100BF00019F4823041F4CBC0843019F4923079F486
:100C0000C6C0923051F481E02A859A89291709F4E7
:100C100080E08A87CE010996BCC0823051F481E021
:100C20002A859A89291709F480E08A8BCE0141969A
:100C3000B0C06D847E848F849888ED88FE880F898B
:100C4000188DE0E2F0E080E090E0DC01AA24BB2413
:100C5000650120E030E0A901B30161707070611599
:100C60007105D1F02E0D3F1D401F511F15012601AA
:100C7000280E391E4A1E5B1E81E090E0A0E0B0E025
:100C80002E153F054007510718F080E090E0DC0189
:100C9000820D931DA41DB51DAA0CBB1CCC1CDD1C14
:100CA00017FF09C061E0262E312C412C512CA228BF
:100CB000B328C428D528319749F0EE0CFF1C001F3B
:100CC000111F9694879477946794C6CF6B897C891B
:100CD000EB85FC856E0F7F1F6E5F7F4F7C8F6B8F68
:100CE00061E0EA857A89E71709F460E06A8F6B8D25
:100CF0007C8D10C0FC01E170F070309729F05695A2
:100D00004795379527955068B695A79597958795F8
:100D10006F5F7F4FB7FDEECF0CC0880F991FAA1FE2
:100D2000BB1F57FD8160220F331F441F551F6150A9
:100D300070408030E0E09E07E0E0AE07E0E4BE07F0
:100D400060F36B8F7C8F6FE7E62EF12C012D112D58
:100D5000E822F9220A231B2360E4E616F1040105C8
:100D6000110561F487FD0AC02115310541055105C2
:100D700029F0805C9F4FAF4FBF4F80788D8F9E8F43
:100D8000AF8FB8A383E0898FCE01499602C081E27C
:100D900091E00E94CF07A096E2E10C948609A8E1B9
:100DA000B0E0E5EDF6E00C94720969837A838B83F9
:100DB0009C832D833E834F8358878E01075F1F4F8F
:100DC000CE010196B8010E949D0881E1E82EF12C28
:100DD000EC0EFD1ECE010596B7010E949D08998577
:100DE000923008F483C08989823008F47BC02A8558
:100DF0003A8923272A87943011F0923021F49817EA
:100E000009F06CC071C0843039F41D861E861F86BF
:100E1000188A1C861B866AC0823019F484E0898790
:100E200065C08B859C852B893C89821B930B9C8795
:100E30008B872D853E854F855889ED88FE880F89E3
:100E4000188D2E153F054007510738F4220F331F28
:100E5000441F551F01979C878B876FE170E0A12C81
:100E6000B12CC12CA0E4DA2E80E090E0DC012E153C
:100E70003F054007510740F08A299B29AC29BD292D
:100E80002E193F09400B510BD694C794B794A794E1
:100E9000220F331F441F551F6150704041F76FE709
:100EA000E62EF12C012D112DE822F9220A231B2315
:100EB00060E4E616F1040105110561F487FD0AC03E
:100EC000211531054105510529F0805C9F4FAF4F39
:100ED000BF4F80788D879E87AF87B88B8E01075F65
:100EE0001F4F04C0870102C001E211E0C8010E9447
:100EF000CF076896EAE00C948E09ACE0B0E0E3E836
:100F0000F7E00C947A0969837A838B839C83CE0102
:100F10000196BE016B5F7F4F0E949D088D818230DC
:100F200081F1823070F1843021F48E81882369F15F
:100F30000AC02F81388537FD24C06E812F313105DD
:100F40003CF0662311F120E030E040E050E821C0A1
:100F50008EE190E0821B930B29853A854B855C8559
:100F600004C056954795379527958A95D2F76623FD
:100F700081F050954095309521953F4F4F4F5F4FF1
:100F800008C020E030E0A90104C02FEF3FEF4FEF91
:100F90005FE7B901CA012C96E2E00C949609EF9242
:100FA000FF920F931F93CF93DF93FC012481358130
:100FB0004681578161818081823020F44061EFEF6A
:100FC000F0E0A3C0843009F49BC0823009F492C0E1
:100FD000211531054105510509F48FC00280F381C7
:100FE000E02D8FEFE238F8070CF05AC0C2E8DFEFCF
:100FF000CE1BDF0BCA31D1056CF579018A010C2EAD
:1010000004C016950795F794E7940A94D2F781E007
:1010100090E0A0E0B0E00C2E04C0880F991FAA1F3A
:10102000BB1F0A94D2F70197A109B1098223932328
:10103000A423B52321E030E040E050E00097A10573
:10104000B10519F420E030E0A9012E293F29402BF9
:10105000512B03C020E030E0A901DA01C9018F77EC
:101060009070A070B07080349105A105B10539F47D
:1010700027FF09C0205C3F4F4F4F5F4F04C0215CEA
:101080003F4F4F4F5F4FE1E0F0E0203080E0380706
:1010900080E0480780E4580728F5E0E0F0E022C04F
:1010A000E038F1056CF5E158FF4FDA01C9018F779F
:1010B0009070A070B07080349105A105B10539F42D
:1010C00027FF09C0205C3F4F4F4F5F4F04C0215C9A
:1010D0003F4F4F4F5F4F57FF05C056954795379588
:1010E0002795319687E056954795379527958A95A8
:1010F000D1F70BC0E0E0F0E005C0E0E0F0E005C0B3
:10110000EFEFF0E020E030E0A9018E2F87958827EF
:101110008795942F9F77679566276795E695E22ECA
:10112000A92FA82BFE2FF62B622F732F8A2F9F2F0C
:10113000CDB7DEB7E6E00C949209DC01FB012C91FF
:1011400011963C91119712968C911297482F4F77D8
:1011500050E0982F991F9927991F13966C91139718
:10116000862F880F892B90E0661F6627661F618394
:10117000009739F5211531054105510511F482E03B
:1011800029C082E89FEF9383828367E0220F331F99
:10119000441F551F6A95D1F783E0808309C0220F51
:1011A000331F441F551F828193810197938382834C
:1011B000203080E0380780E0480780E4580778F363
:1011C00020C08F3F910579F4211531054105510566
:1011D00019F484E08083089544FF03C081E0808394
:1011E00010C010820EC08F5790409383828383E09B
:1011F000808387E0220F331F441F551F8A95D1F744
:1012000050642483358346835783089597FB092EC2
:1012100007260AD077FD04D049D006D000201AF462
:10122000709561957F4F0895F6F7909581959F4F42
:101230000895A1E21A2EAA1BBB1BFD010DC0AA1F17
:10124000BB1FEE1FFF1FA217B307E407F50720F02F
:10125000A21BB30BE40BF50B661F771F881F991FAA
:101260001A9469F760957095809590959B01AC01F3
:10127000BD01CF01089597FB092E05260ED057FD1D
:1012800004D0D7DF0AD0001C38F450954095309533
:1012900021953F4F4F4F5F4F0895F6F790958095FA
:1012A000709561957F4F8F4F9F4F0895AA1BBB1B71
:1012B00051E107C0AA1FBB1FA617B70710F0A61B56
:1012C000B70B881F991F5A95A9F780959095BC0177
:1012D000CD0108952F923F924F925F926F927F922D
:1012E0008F929F92AF92BF92CF92DF92EF92FF9236
:1012F0000F931F93CF93DF93CDB7DEB7CA1BDB0BE2
:101300000FB6F894DEBF0FBECDBF09942A88398886
:1013100048885F846E847D848C849B84AA84B9848D
:10132000C884DF80EE80FD800C811B81AA81B98199
:10133000CE0FD11D0FB6F894DEBF0FBECDBFED01AD
:101340000895EE0FFF1F0590F491E02D09949F93EF
:1013500005D00F9007FCEE5F28C0CEC03FD0E8F369
:10136000E894E0E0BB279F57F0F02AED3FE049EC1E
:1013700006C0EE0FBB0F661F771F881F28F0B23A1A
:1013800062077307840728F0B25A620B730B840B51
:10139000E3959A9572F7803830F49A95BB0F661FE3
:1013A000771F881FD2F790489BC0EF93E0FF06C0DD
:1013B000A2EA2AED3FE049EC5FEB37D0BFD00F90B7
:1013C000039401FC9058E8E6F0E099C057FD90586E
:1013D000440F551F59F05F3F71F04795880F97FBF9
:1013E000991F61F09F3F79F08795089512161306B3
:1013F0001406551FF2CF4695F1DF08C016161706E2
:101400001806991FF1CF8695710561050894089516
:1014100087D030F08CD020F031F49F3F11F41EF4CF
:101420006BC00EF4E095E7FB53C0E92FCFDF80F3EC
:10143000BA17620773078407950718F071F49EF5D1
:101440008EC00EF4E0950B2EBA2FA02D0B01B90122
:1014500090010C01CA01A0011124FF27591B99F02A
:10146000593F50F4503E68F11A16F040A22F232F36
:10147000342F4427585FF3CF469537952795A79586
:10148000F0405395C9F77EF41F16BA0B620B730B2D
:10149000840BBAF09150A1F0FF0FBB1F661F771F9E
:1014A000881FC2F70EC0BA0F621F731F841F48F453
:1014B000879577956795B795F7959E3F08F0B3CFD9
:1014C0009395880F08F09927EE0F979587950895C3
:1014D00097F99F6780E870E060E008959F3F31F0E2
:1014E000915020F4879577956795B795880F911D52
:1014F0009695879597F908959FEF80EC08959F93AF
:101500008F937F936F93FF93EF939B01AC014DDB20
:10151000EF91FF912BD02F913F914F915F9145CB50
:1015200000240A94161617061806090608950024C2
:101530000A9412161306140605060895092E03943C
:10154000000C11F4882352F0BB0F40F4BF2B11F4B0
:1015500060FF04C06F5F7F4F8F4F9F4F0895E894E7
:10156000BB2766277727CB0197F90895DF93CF93A1
:101570001F930F93FF92EF92DF927B018C0168948F
:1015800005C0DA2EEF0121D0FE01E894A591259146
:10159000359145915591AEF3EF0147DFFE0197017B
:1015A000A801DA9479F7DF90EF90FF900F911F91E7
:1015B000CF91DF910895B4DF28F0B9DF18F09523BB
:1015C00009F086CF99CF1124CBCF00DFA0F3959FF0
:1015D000D1F3950F50E0551F629FF001729FBB271A
:1015E000F00DB11D639FAA27F00DB11DAA1F649FC6
:1015F0006627B00DA11D661F829F2227B00DA11D79
:10160000621F739FB00DA11D621F839FA00D611DFE
:10161000221F749F3327A00D611D231F849F600D1F
:10162000211D822F762F6A2F11249F5750408AF058
:10163000E1F088234AF0EE0FFF1FBB1F661F771FE4
:10164000881F91505040A9F79E3F510570F040CF40
:1016500087CF5F3FECF3983EDCF3869577956795EF
:10166000B795F795E7959F5FC1F7FE2B880F911D02
:0C1670009695879597F90895F894FFCFA0
:10167C0057656C636F6D6520746F20656C65637462
:10168C006963000E0F10111213141500000000D521
:0A169C000100000000000000000043
:00000001FF
